:100000007A2A0000000000000000FF3E031C0800E8
:100010000528FF3E031908000928FB3E03180D2898
:1000200008001220132000308C004E3001208C0B71
:10003000152808008D0011208D0B1B280800831641
:100040000814831208080800880083160815553024
:100050008900AA308900881488182C288312081176
:1000600008000E08850008000F08860008008E149E
:1000700031288E1031289014100865000800901067
:100080001008650008000E1531280E1131281015D2
:1000900010086500080010111008650008008E1592
:1000A00031288E1131280E1631280E1231281016E3
:1000B00010086500080010121008650008000F14F1
:1000C00034280F10342804308F06342811151108F5
:1000D00066000800111111086600080008308F063C
:1000E0003428911511086600080091111108660066
:1000F00008000F1634280F12342811161108660054
:10010000080011121108660008008F1634288F129B
:100110003428911611086600080091121108660033
:1001200008000F1734280F13342811171108660020
:10013000080011131108660008008F1734288F1368
:100140003428911711086600080091131108660001
:10015000080004308F060F08860008308F060F084D
:1001600086000800A7146A207520BA28A710662008
:100170007120BA2810309200A920920BBC280800E8
:100180009300C420C420C4204B2037200E11131824
:100190000E153120930CA9203920A920A920080090
:1001A0009301D420D420D4203720930C9311A9207C
:1001B000051993153920A920A92013080800C0208B
:1001C0009301C32008001310C4201C08C0201B0882
:1001D000C0201A08C02019089300C3201310C4209F
:1001E00008004720D420D02021059C00D0202005E5
:1001F0009B00D0201F059A00D320930C130C1E05E2
:100200009900D4204B200800143097000A21970B46
:100210000629080064309600BA20960B0C290800C5
:100220005520BA2053200800B62004213B20472047
:1002300010210800612014213F2047201021572061
:100240009701050D8500051C2029960B2129970B88
:10025000212953205B204F20080003309E000F30DF
:100260009F000F30A0000F30A100080000309E005A
:1002700000309F000F30A0000F30A10008002D219A
:1002800002309500043094000800362103309500B8
:100290000530940008002D210230950004309400B0
:1002A00004210030DF20E3200800033099000F30E4
:1002B0009A000F309B000F309C000030DF20E320BD
:1002C00007309600E221960B62290130DF200730CB
:1002D000DF200830DF200A210130DF200730DF2057
:1002E00010210030990000309A000F309B000F3031
:1002F0009C000330DF20E3200830DF200A210B3090
:10030000DF200830DF200A210800392045203F2067
:100310004B20B220042110210A211C080C3C031997
:100320003F211C080D3C031945211C080F3C0319F3
:100330004B211C080E3C0319552108001408DF202E
:10034000F1200800190822069906A2061A082306B9
:100350009A06A3061B0824069B06A4061C0825066D
:100360009C06A5060800190822061E053F30031D3D
:100370009D001A0823061F053F30031D9D001B0822
:10038000240620053F30031D9D001C08250621057D
:100390003F30031D9D0008001508DF20E3200830D2
:1003A000DF200A21A2219E21B3210800A2219E2143
:1003B000B3211D083F3A031D08004C309D00A221C7
:1003C000CC2108000630DF2008001808F63E03188C
:1003D000073E3A3E9D0008007D2089209520A120FF
:1003E0008F131C188F1734200F139C180F173420ED
:1003F0008F121C198F1634200F129C190F163420DF
:100400001B18A5209B1899201B198D209B19812052
:100410000800190E1A0489001B0E1C042420080071
:100420001B0E1C0489001F2008080F399A00080EB3
:100430000F39990008000030990002309A0000300E
:100440009B0000309C0008002030990012309A0078
:100450001C309B0019309C00080000301906031D59
:10046000080000301A06031D080000301B06031D9B
:10047000080000301C06031D08002714080089012D
:100480001F2019080806031D0800890A1F201A08E2
:100490000806031D0800890A1F201B080806031D03
:1004A0000800890A1F201C080806031D0800890A85
:1004B0002714080027102D223F220800890119085F
:1004C0002420890A1A082420890A1B082420890A62
:1004D0001C082420080089011F209900890A1F2078
:1004E0009A00890A1F209B00890A1F209C0008008F
:1004F00027100800F73090006500FE30910066007C
:100500007D2089209520A1205B2053206320B620E8
:100510002714A7106120C83014205F2004308F06F4
:100520000F08860008308F060F0886000310051C90
:10053000A82AA9011730A800051CFF3EA80B9C2A79
:10054000E83E0C3EA90C031C0319A72A9A2A290984
:10055000031C8E2A9D009F3E03189D122718B52A62
:100560001D08483C03195A22F92A1D08473C031963
:1005700014211D08483C03195A221D08493C03193F
:10058000E2211D084C3C0319D6211D084D3C0319DE
:1005900009221D084B3C031910221D08503C031969
:1005A0001A211D08513C03196B221D08523C0319E6
:1005B0009E211D08533C031978221D08543C031941
:1005C00024221D08553C03195E221D08563C0319C0
:1005D0001B221D08573C0319CC211D08583C031948
:1005E00085211D085A3C0319EC211D084E3C0319B6
:1005F000E521190898001A0899001B089A001C08A0
:100600009B001D08BF3E0318F93E113E9C002718B1
:100610000D2B5F2006300120962AA60A0F14261BF8
:100620000F1034201D081523962AAA000A30AB00AB
:100630004F20153003202A1851202A1C4F20AA0CC5
:08064000AA17AB0B192B0800EF
:02400E00FA3F77
:00000001FF
